:0900000002000EB2EF32B2EE3242
:0F000B00020003787FE4F6D8FD75810D020080B6
:10001B00020006EFD3940174809480500EEFC4332A
:10002B003354C0FFE5AF54BF4FF5AFE4FF22EFD31E
:10003B00940174809480500DEF25E025E0FFE5AF2F
:10004B0054FB4FF5AFE4FF227509F8E4F508FB7A92
:10005B000079087F060200A602008AEFD394017490
:10006B00809480500DEFC43354E0FFE5AF54DF4F65
:10007B00F5AFE4FF22120053120580D2AF80FEB21F
:08008B00ED32B2EC32B2EB32AF
:03009B0002008DD3
:1000A300020090EFD394077480948040037FFF2273
:1000B300120623FED394037480948040037FFF22AF
:1000C300EF7044EE700B90000112063CF452935211
:1000D300941206236401700B90000112063C4293B4
:1000E300F45294120623FE6402700A900001120671
:1000F3003C42934294EE6403700D90000112063C5F
:10010300FEF45293EE4294EF64017046120623FE0E
:10011300700B90000112063CF452915292EE64016E
:10012300700B90000112063C4291F4529212062386
:100133006402700A90000112063C42914292120638
:10014300236403700D90000112063CFEF45291EEFD
:100153004292EF64027046120623FE700B90000178
:1001630012063CF452955296EE6401700B90000116
:1001730012063C4295F452961206236402700A90CA
:10018300000112063C429542961206236403700D49
:1001930090000112063CFEF45295EE4296EF640382
:1001A3007046120623FE700B90000112063CF452B7
:1001B300B152B2EE6401700B90000112063C42B1E1
:1001C300F452B21206236402700A90000112063C34
:1001D30042B142B21206236403700D90000112066D
:1001E3003CFEF452B1EE42B2EF64047046120623B1
:1001F300FE700B90000112063CF452B352B4EE644D
:1002030001700B90000112063C42B3F452B4120683
:10021300236402700A90000112063C42B342B412F6
:1002230006236403700D90000112063CFEF452B3E2
:10023300EE42B4EF64057046120623FE700B900085
:100243000112063CF452C952CAEE6401700B9000CD
:100253000112063C42C9F452CA1206236402700A10
:1002630090000112063C42C942CA1206236403707D
:100273000D90000112063CFEF452C9EE42CAEF642F
:10028300067046120623FE700B90000112063CF422
:1002930052CB52CCEE6401700B90000112063C422B
:1002A300CBF452CC1206236402700A9000011206AA
:1002B3003C42CB42CC1206236403700D9000011222
:1002C300063CFEF452CBEE42CCEF640770491206B3
:1002D30023FF7E00700B90000112063CF452E152A2
:1002E300E2EF64014E700B90000112063C42E1F410
:1002F30052E21206236402700A90000112063C4285
:10030300E142E21206236403700D90000112063CE1
:10031300FFF452E1EF42E27F0022AD07ED707EC2AF
:100323008C120623FEC394037480948040037FFFE2
:1003330022E58954FC4EF58990000112063CFED358
:1003430094027480948040037FFF22EEFF7E00704E
:1003530006538E7F5389FBEF64014E7006438E80F4
:100363005389FBEF64024E70034389049000021229
:10037300063CFFE58F54FE4FF58F9000031206698C
:10038300E5F0F58C900003120669F58A90000512DA
:10039300063C7004C28C8002D28C7F0022ED640183
:1003A300600302042DC28E120623FEC394037480DD
:1003B300948040037FFF22EEC454F0FFE58954CFBD
:1003C3004FF58990000112063CFED3940274809489
:1003D3008040037FFF22EEFF7E007006538EBF53E3
:1003E30089BFEF64014E7006438E405389BFEF64AB
:1003F300024E700343894090000212063C25E0FF41
:10040300E58F54FD4FF58F900003120669E5F0F573
:100413008D900003120669F58B90000512063C705F
:1004230004C28E8002D28E7F0022ED64027061537B
:100433008EEF90000112063CFF7E007006538EFB88
:10044300538EF7EF64014E7006438E04538EF7EF1D
:1004530064024E7003438E0890000212063C25E0AE
:1004630025E0FFE58F54FB4FF58F900003120669DB
:10047300E5F0F5D6900003120669F5D79000051252
:10048300063CC454F0FFE58E54EF4FF58E7F0022F7
:10049300ED6403706953D1F790000112063CFED35B
:1004A30094027480948040037FFF22EEFF7E0070ED
:1004B3000653D1FD53D1FBEF64014E700643D102C5
:1004C30053D1FBEF64024E700343D1049000021238
:1004D300063CFFE5D154FE4FF5D1900003120669A7
:1004E300E5F0F5D4900003120669F5D590000512E6
:1004F300063C33333354F8FFE5D154F78076ED648B
:1005030004707753D17F90000112063CFD7C00D329
:1005130094027480948040037FFF22ED4C70065355
:10052300D1DF53D1BF90000112063C640170064332
:10053300D12053D1BF90000112063C6402700343E3
:10054300D14090000212063CC454F0FFE5D154EFB1
:100553004FF5D1900003120669FDACF0ECF5D2AF74
:10056300058FD390000512063CC43333335480FF08
:10057300E5D1547F4FF5D17F00227FFF22E4F508B8
:10058300750901F50A750BFF750C10750D01FB7AE2
:10059300007908FF12031DE4FD7F011206A1E4F5B3
:1005A30008750901F50A750BF6750CA0750D01FBAD
:1005B3007A0079087F0112031DE4FD7F011206EE24
:1005C300750901E4F50A750BA2750C40750D01FB65
:1005D3007A0079087F0212031DE4FD7F01120039BE
:1005E300E4F509750A01750BB1750CE0750D01FB96
:1005F3007A0079087F0312031DE4FD7F0112006670
:10060300E4F509750A01750B63750CC0750D01FBE3
:100613007A0079087F0412031DE4FD7F0102001EA6
:10062300BB010689828A83E0225002E722BBFE02D5
:10063300E32289828A83E49322BB010CE58229F5B4
:1006430082E5833AF583E0225006E92582F8E62223
:10065300BBFE06E92582F8E222E58229F582E583DD
:100663003AF583E49322BB0110E58229F582E58301
:100673003AF583E0F5F0A3E0225009E92582F886F4
:10068300F008E622BBFE0AE92582F8E2F5F008E26B
:1006930022E5832AF583E993F5F0A3E99322EFFB9F
:1006A300D39401748094805009EB7004C2A9800232
:1006B300D2A9EDFF7E00D39403748094805029EF78
:1006C300700553B7FDC2B9EF64014E700553B7FD12
:1006D300D2B9EF64024E700543B702C2B9EF6403A7
:1006E3004E700543B702D2B97F0022EFFBD39401CA
:1006F300748094805009EB7004C2AB8002D2ABEDDE
:10070300FF7E00D39403748094805029EF700553C7
:10071300B7F7C2BBEF64014E700553B7F7D2BBEF17
:1007230064024E700543B708C2BBEF64034E700505
:0807330043B708D2BB7F00228E
:00000001FF
